:0A0000000C9493030C9400000C9480
:10000A0000000C9400000C9400000C9400000C9466
:10001A0000000C9400000C9400000C947A100C94CC
:10002A0000000C946A0A0C9400000C94DE110C94E3
:10003A0000000C9400000C9400000C9400000C9436
:10004A0000000C9400000C9400000C9400000C9426
:10005A0000000C9400000C940000000204060A0E32
:10006A0012161A1E22262A2E32363A3E42464A00D4
:10007A002020205330372F56322E33332020202091
:10008A000000DCDCDCDCDCDCDCDCDCDCDCDCDCDC5E
:10009A00DCDCDCDCDCDCDCDCDCDCDCDCDCDCDCDC96
:1000AA00DCDCDCDCDCDCDCDCDCDCDCDCDCDCDCDC86
:1000BA00DCDCDCDCDCDCDCDCDCDCDCDCDCDCD6D484
:1000CA00D3D2D0CFCECCCBCAC8C7C6C5C4C2C1C092
:1000DA00BFBEBDBCBAB9B9B8B7B6B4B3B2B1B1B0A4
:1000EA00AFAEADACABAAA9A8A7A7A6A5A4A3A2A187
:1000FA00A09F9F9E9C9B9B9A99999897969594935B
:10010A00929191908F8F8E8D8C8B8B8A898887861E
:10011A0085858482818180807F7E7D7D7C7B7A79E2
:10012A0078777675757473727170706F6E6D6C6BAB
:10013A006A696867676664636261605F5E5D5C5B8B
:10014A005A5958575655545352504F4E4D4C4A4986
:10015A0048464442403E3D3C39363432302E2C2A01
:10016A00281E1C1B1A19171514131211100F0E0D25
:10017A000C0B0A0908070605040302010000000027
:10018A000000D5DBD5DBE3E7E3E7EAEDEAED88F14A
:10019A0088F1D9F2D9F2F2F3F2F3DFF4DFF4AAF537
:1001AA00AAF55BF65BF6F5F6F5F67DF77DF7F6F759
:1001BA00F6F763F863F8C4F8C4F81CF91CF96CF98B
:1001CA006CF9B6F9B6F9F9F9F9F937FA37FA6FFAB3
:1001DA006FFAA4FAA4FAD5FAD5FA03FB03FB2DFBAE
:1001EA002DFB55FB55FB7BFB7BFB9EFB9EFBBFFB65
:1001FA00BFFBDEFBDEFBFBFBFBFB17FC17FC31FC4A
:10020A0031FC4AFC4AFC62FC62FC79FC79FC8EFCFB
:10021A008EFCA3FCA3FCB6FCB6FCC9FCC9FC020319
:10022A000405060708090A0B0C0D0E0F101112130C
:10023A001415160000011027E80364000A000100E3
:10024A000010000110000100253033640020205402
:10025A000020202D2D2D2057414954202D2D2D20B1
:10026A00200020202020205265616479202020204F
:10027A002020002020204C414D494E41544F52200D
:10028A002020200025303464202020202020202017
:10029A00202020200020202D2D2D2042555359208A
:1002AA002D2D2D20200020496E697469616C697AB0
:1002BA006174696F6E20002E2E2E2E2E2020202093
:1002CA0020203030302E43002020202020202020E3
:1002DA00202020202020202000233633204F757430
:1002EA0020746F205072692E2E0023363420456AFE
:1002FA0065637420202020202020002336352054D6
:10030A0072616E73706F727420202000233636205B
:10031A0052657472616374202020202000233637CE
:10032A002066696C6D20696E64657820200023362A
:10033A003920656E64206F662066696C6D20002323
:10034A003833204144432070726F626C656D20001F
:10035A00233834206865617420726F6C6C65722072
:10036A00002338362053656E736F72203F3F3F205B
:10037A0020004C616D696E6174696F6E20537065FF
:10038A006564004C616D696E6174696F6E205370AB
:10039A006565642020202020202020202020202085
:1003AA002020202020202020202020202020202043
:1003BA002020202020202020202020202020202033
:1003CA002020202020202020202020202020202023
:1003DA00202020005072652D4C616D692E204465E5
:1003EA006C617920005072652D4C616D692E204434
:1003FA00656C6179202020202020202020202020C8
:10040A0020202020202020202020202020202020E2
:10041A0020202020202020202020202020202020D2
:10042A0020202020202020202020202020202020C2
:10043A002020202020002020456E6420506F736900
:10044A0074696F6E2020002020456E6420506F73FF
:10045A006974696F6E20202020202020202020200F
:10046A002020202020202020202020202020202082
:10047A002020202020202020202020202020202072
:10048A002020202020202020202020202020202062
:10049A0020202020202020002053746172742050D4
:1004AA006F736974696F6E200020537461727420CF
:1004BA00506F736974696F6E2020202020202020DD
:1004CA002020202020202020202020202020202022
:1004DA002020202020202020202020202020202012
:1004EA002020202020202020202020202020202002
:1004FA0020202020202020202020004C616D696EC1
:10050A006174696F6E4C656E677468004C616D69E1
:10051A006E6174696F6E4C656E6774682020202066
:10052A0020202020202020202020202020202020C1
:10053A0020202020202020202020202020202020B1
:10054A0020202020202020202020202020202020A1
:10055A0020202020202020202020202000202020B1
:10056A00204F5054494F4E532020202020004D4503
:10057A004E5520205341564520202020202020205F
:10058A002020202020202020202020202020202061
:10059A002020202020202020202020202020204F22
:1005AA005645524C4159202020202020202020202E
:1005BA002020202020202020202020202020002051
:1005CA0020504154434800202020202020544553E5
:1005DA005420202020202000206463312A202E2E3F
:1005EA002E2E20204D454E55202020202020202030
:1005FA0020202020202020202020202020202020F1
:10060A002064633220202064633320204D4F44301D
:10061A0020202020202020202020202020202020D0
:10062A002020202020202020004D4F4430004D4F14
:10063A004431004D4F4432004D4F4433002044436F
:10064A00312A00202020205341564520414C4C207D
:10065A0020202000202020504152414D455445522F
:10066A0020202020004F5645524C415900206463F7
:10067A00312A0020646332200020444332200020C3
:10068A0064633320002044433320002020202025A7
:10069A0064206D6D2F732020202020002020202030
:1006AA002564206D73202020202020202020202057
:1006BA0020002020202564206D6D2020202020206D
:1006CA00202020202020202020002D3E20256420CC
:1006DA007820312F35306D6D202020003C2D2025CB
:1006EA0064207820312F35306D6D202020002020A5
:1006FA00202564207820312F35306D6D2020200090
:10070A00310D00300D0025750D0025640D002530D2
:10071A0032580D00330D00320D000000F894EE2718
:10072A00EFBBF1E0FBBFEBBFE5BFF8E1F093600080
:10073A00E09360008DE0A2E0BB27ED938A95E9F78C
:10074A0080E098E0A0E0B1E0ED930197E9F7E4E2F8
:10075A00F7E085919591009761F0A591B591059083
:10076A001590BF01F00105900D920197E1F7FB0189
:10077A00F0CFE0E0EEBBE0E0EABDE0E0EBBDEFEF9A
:10078A00EDBFE8E0EEBFC0E0D3E00C94CC032A97BB
:10079A003DD40E946C13FE01FA93EA93E2E5F2E07B
:1007AA00FA93EA93E091F104FF27662777270E94DC
:1007BA00BF2384E00E9404202896EBE4F5E00E941F
:1007CA008420E091F404EA931ED6E093F204EAB599
:1007DA00E5FF17C0FE01FA93EA93E2E5F2E0FA9325
:1007EA00EA93E091F204FF27662777270E94BF2346
:1007FA0084E00E9404202896E7E4F5E00E94842021
:10080A000CC0E7E4F5E0FA93EA93E7E5F2E0FA933D
:10081A00EA93E3E0EA930E946B23A0911305A030C8
:10082A0021F4A0918805A03009F01AC0A0917105A1
:10083A00A03019F0EBB5E0FF13C031FE07C0E8E1C4
:10084A00F5E0FA93EA93EBE5F2E006C0E8E1F5E0B9
:10085A00FA93EA93ECE6F2E0FA93EA930E948E2086
:10086A000E94941AE0918E05E03021F4E0918F0500
:10087A00E03009F025C3E0917105A0917005EA17EF
:10088A0040F4DDD4E0917005E0937105E0E0E09377
:10089A007005E0917105E03061F04B990AC0A091B2
:1008AA001605B09117050E94C42319F4EBB5E1FFB0
:1008BA0002C056FE2DC0A0917105A33409F423C0CD
:1008CA00A0917105A53419F4E89422F81CC0A091EE
:1008DA007105AF3341F4E091DB00E17019F0EFE408
:1008EA00E093700513C0A0917105A13409F40BC0FF
:1008FA00A0917105E2E0EA1710F4A83208F006C0E8
:10090A00E0E0E0937105EFE4E0937005E89456F8AF
:10091A004D9902C032FE01C024C0E2E3E093CC0448
:10092A000E949220E9E1E0936F050E94982008F462
:10093A00FCCFE0E0E093CD044D990AC0EEE0F1E08F
:10094A00E093D004F093D1040E949D20F49AF4CF4E
:10095A00EAE0E0936F050E94982008F4FCCFF4992E
:10096A00FECF4A990EC0E0917B05E17051F0A0914B
:10097A001605B09117050E94C42319F4EBB5E1FFDF
:10098A0001C029C0A091F104A43B78F4E091F104DC
:10099A00EF5FE093F104E150E091F1040E94A1209D
:1009AA00E093F304E4E6E0936E05EAE0E0936F0572
:1009BA000E94982008F4FCCF4A9904C0E0917A0575
:1009CA00E03009F401C0F8CFEAE0E0936F050E9435
:1009DA00982008F4FCCF4E990EC0E0917B05E17097
:1009EA0051F0A0911605B09117050E94C42319F47D
:1009FA00EBB5E1FF01C02AC0A091F104E4E6EA17D1
:100A0A0078F4E091F104E150E093F104EF5FE091B2
:100A1A00F1040E94A120E093F304E4E6E0936E055A
:100A2A00EAE0E0936F050E94982008F4FCCF4E9903
:100A3A0004C0E0917A05E03009F401C0F8CFEAE099
:100A4A00E0936F050E94982008F4FCCF4F9910C0DC
:100A5A0032FC0EC0E0917B05E17051F0A0911605C1
:100A6A00B09117050E94C42319F4EBB5E1FF01C048
:100A7A0065C0EDE7F2E00E94A520EBB5E2FF17C0E2
:100A8A00E3E4F3E0FA93EA93EEE8F2E0FA93EA9306
:100A9A00E0913703F0913803662777270E94BF2336
:100AAA0084E00E9404202896E0E2E0935303E9E1FF
:100ABA00E0936F050E94982008F4FCCF4F9937C045
:100ACA004A9919C0EAB5E5FF03C0EAB5EF7D02C04D
:100ADA00EAB5E062EABDEAE0E0936F050E94982079
:100AEA0008F4FCCF4A9BFECFEAE0E0936F050E9430
:100AFA00982008F4FCCF4E9919C0EBB5E2FF03C069
:100B0A00EBB5EB7F02C0EBB5E460EBBDEAE0E09346
:100B1A006F050E94982008F4FCCF4E9BFECFEAE0B6
:100B2A00E0936F050E94982008F4FCCFC7CFEAE053
:100B3A00E0936F050E94982008F4FCCF4C9910C0EE
:100B4A0032FC0EC0E0917B05E17051F0A0911605D0
:100B5A00B09117050E94C42319F4EBB5E1FF01C057
:100B6A0006C0689433F80E944515E89433F8E0917A
:100B7A008805E03009F4E0D1E091DB00E17009F486
:100B8A00A1D1E0918805E03041F5F59B06C021FC32
:100B9A0004C0A0918905A03009F01EC0E8E1F5E083
:100BAA00FA93EA93EFE9F2E0FA93EA930E948E202D
:100BBA00E0917B05E27071F0E0917B05E47029F425
:100BCA00689436F8EFE7E0934405E1E0E09389059D
:100BDA00EAE074C10E94B12073C1E130A1F4E0914E
:100BEA007B05E07151F02C9AE8ECE0936D05E2E3A5
:100BFA00F0E0E093E804F093E904E0918805EF5F00
:100C0A00E09388055DC1E23051F5E0917B05E07122
:100C1A0019F1E091DB00E870E1F4EAEFE0936F0587
:100C2A000E94982008F4FCCFEAEFE0936F050E9437
:100C3A00982008F4FCCFE091DB00E87039F4E3E493
:100C4A00E09370052C98F598E4E138C10E94B12030
:100C5A0002C00E94B12002C00E94B12031C1E3301B
:100C6A0041F5E0917B05E07109F1E091DB00E87064
:100C7A0021F42C980E94B72018C0A0916D05A530C8
:100C8A0038F4E3E4E09370052C98F598E4E116C192
:100C9A00E091E804F091E904309739F4E5E4E0934F
:100CAA0070052C98F598E4E109C102C00E94B720AA
:100CBA0007C1E430C1F4E0918305E03099F420FCE7
:100CCA0009C0E091ED04EE0FEE5FE0936D050E941E
:100CDA00B12008C0E1E0E0938605F598E4E5E093E9
:100CEA007005EBC0EDC0E53081F4A0916D05A2302E
:100CFA0028F4E2E3E093CC040E949220A0916D05CF
:100D0A00A13010F40E94B120DBC0E63011F00C943F
:100D1A00CD060091CA0473D1E0E2FAE0E093E6045A
:100D2A00F093E704E89422F8E8E3F4E0E093D804C7
:100D3A00F093D904E0917B05E07131F0ECE6F0E044
:100D4A00E093D804F093D904E091DA00E860E093E4
:100D5A00DA00E2E3E093CC040E949220A091D4044A
:100D6A00B091D504E2E0F0E00E949C23E25AF04000
:100D7A00E093D004F093D1040E949D20F49A6894E1
:100D8A0035F8E6E7E0934405E0918805EF5F96C001
:100D9A00E73049F5F4990AC00093CA040E94BB20BF
:100DAA00E89435F8E0918805EF5F1AC022FE1AC070
:100DBA00E5E4E0937005ECE6F0E0E093D004F0930C
:100DCA00D1040E949D20F49AE0E0F0E0E093D80478
:100DDA00F093D9042C980093CA040E94BB20E4E142
:100DEA00E09388056DC0E83021F4E0918805EF5F53
:100DFA0065C0E930C9F4E091EE040E94C420E09392
:100E0A00D604F093D704E2E3E093CC040E94922044
:100E1A00E1E0E0938905689436F8EFE7E09344054A
:100E2A00E0918805EF5F4AC0EA3011F5E091890543
:100E3A00E030E9F42C98E0917B05E47041F0A09150
:100E4A007005A03021F4A0917105A03009F00CC002
:100E5A00689436F8EEE7E0934405E1E0E0938A050A
:100E6A00E0918805EF5F01C0E0E0E093880528C0C3
:100E7A00EB3041F4E0918A05E03019F4E0E0E093C8
:100E8A0088051EC0E431B1F4E0918605E03089F4AA
:100E9A00E2E3E093CC040E949220E8EFF5E2E093CB
:100EAA00D004F093D1040E949D20F49AE3E6E093E3
:100EBA00880506C0F49904C02C98E0E0E093880500
:100ECA006ACCFFCF21FC0895F6990895F69AF59910
:100EDA000895E0919005E03009F00895689432F899
:100EEA00E1E2E0934305E0E0F0E0E093D204F0931E
:100EFA00D304E2E3E093CC040E949220E9E1E09378
:100F0A006F050E94982008F4FCCFE1E0E093900579
:100F1A00E0E0E093CD04ECE1F2E0E093D004F0935A
:100F2A00D1040E949D20F49AEFE0E0936F050E949D
:100F3A00982008F4FCCF0895E091DB00E17021F0DD
:100F4A00E091DB00E27009F41EC0E0919005E03008
:100F5A0049F0A091CE04B091CF04EEE0F1E0EA1797
:100F6A00FB0708F00CC0E0E0E0939005E8EDF0E044
:100F7A00E093D004F093D1040E949D20F49AE0E01B
:100F8A00E0939005F598E0919005E03071F4F599B9
:100F9A000CC0A0918805A03041F4A0918605A0302C
:100FAA0021F4A0918305A03009F00895E89432F85D
:100FBA0035F836F834F8EEE2E0934405E093430559
:100FCA00E091DB00E17041F0F698A0917105A2343E
:100FDA0019F4EFE4E0937005E091DB00E27009F4A4
:100FEA00F69AE091DB00E47041F0A0917105A0341B
:100FFA0019F4EFE4E093700501C0F69A0895A4E6A7
:10100A00B0E00E94CA20E093CA0408950E94C9234E
:10101A00E0E0E5BFE0E7E2B9EFE8E1B9E1E8E5B928
:10102A00E0E7E4B9E0E0E8B9EFEFE7B9EBB9E0E00F
:10103A00EAB9ECE6EEB9E8E9EDB9ECE0E1BBE0E0EB
:10104A00E0BBEFE1E4BBE0E0E3BBE3ECE093DA0012
:10105A00EFE3E093D900EFE7E093DD00E0E0E0930F
:10106A00DC00E5E0E4BDE4E6E6BDE0E0E093800014
:10107A00E0918100E260E0938100E0E6F0EFE09326
:10108A008400F0938500E0E0E093B000E093B200C2
:10109A00E093B30013E320E0E8E1E093C100E6E067
:1010AA00E093C200E22FF070E093C500E12FF22F27
:1010BA00F070E093C4000091C600E091C100E068BE
:1010CA00E093C100E7E8E0937A00E1E2E0937C0074
:1010DA00139A1298119A119838EC40E000240316DA
:1010EA00040618F431504040F9CFE8E3E8B9139800
:1010FA00139A38EC40E000240316040618F4315021
:10110A004040F9CFE1E0E8B91398139A38E843E18F
:10111A0000240316040618F431504040F9CFEEE0DB
:10112A00E8B91398139A38EC40E000240316040631
:10113A0018F431504040F9CFE6E0E8B91398139A11
:10114A0038EC40E000240316040618F431504040FD
:10115A00F9CFE0E8E8B91398139A119AE0E0EDBBE9
:10116A00E0936900E0916E00E160E0936E00E09127
:10117A006F00E160E0936F00E0E0E09370000E948E
:10118A00D02325960895E091C000E072E1F3E8814A
:10119A00E093C60021960895F894F999FECFE98163
:1011AA00FA81F2BDE1BDE881E0BDFA9AF99A789434
:1011BA0023960895F894F999FECFE881F981F2BD52
:1011CA00E1BDF89A7894E0B5229608950E94CB235F
:1011DA0018E125E000E0003550F4E02FA12FB22FEE
:1011EA00F0E0AE0FBF1FE0E2EC930F5FF4CFA12F48
:1011FA00B22FA05BBF4FE0E0EC93E8E1F5E0FA9391
:10120A00EA93E0EBF2E0FA93EA930E948E20E0E49C
:10121A00F5E0FA93EA93E1ECF2E0FA93EA930E949A
:10122A008E20EFEDE0934E05A0918205A13019F4CE
:10123A00EDE4E09340050E94D22323960895A091FD
:10124A007005AF3419F4E0E0E0937005A0917005E1
:10125A00AA3038F4E89421F8F19810980E94D12025
:10126A0039C0A0917005A83240F4F19AE0E0F2E0AA
:10127A00E093C504F093C6042DC0A0917005A03573
:10128A00B0F4F19AE0E8F0E0E093C504F093C60404
:10129A00E0E0F0E0E093CE04F093CF042C98F598C8
:1012AA000E94D520E0934405689421F813C0A091C8
:1012BA007005A43678F4109AE0E0F0E0E093CE04EA
:1012CA00F093CF042C98F5980E94D520E09344051A
:1012DA00689421F8A0917005ECE3EA1718F4EAB5CE
:1012EA00EE7FEABDE0917005E03039F4E8E1F5E01F
:1012FA00FA93EA93E2EDF2E065C0EBB5E0FD66C071
:10130A00A0917005AF3339F4E8E1F5E0FA93EA9376
:10131A00E3EEF2E057C0A0917005A03439F4E8E199
:10132A00F5E0FA93EA93E4EFF2E04CC0A09170057D
:10133A00A13439F4E8E1F5E0FA93EA93E5E0F3E061
:10134A0041C0A0917005A23439F4E8E1F5E0FA93BE
:10135A00EA93E6E1F3E036C0A0917005A33439F4CC
:10136A00E8E1F5E0FA93EA93E7E2F3E02BC0A09113
:10137A007005A53439F4E8E1F5E0FA93EA93E8E375
:10138A00F3E020C0A0917005A33539F4E8E1F5E057
:10139A00FA93EA93E9E4F3E015C0A0917005A43545
:1013AA0039F4E8E1F5E0FA93EA93EAE5F3E00AC0F2
:1013BA00A0917005A63551F4E8E1F5E0FA93EA93B5
:1013CA00EBE6F3E0FA93EA930E948E200895E3E4B1
:1013DA00F3E0FA93EA93EE81FF81FA93EA930E948B
:1013EA008E20EBE6F3E0FA93EA93EC81FD81FA931F
:1013FA00EA930E948E20E881F981E0931405F09324
:10140A001505269608950A93ACE8B0E0E981F0E064
:10141A00EA0FFB1F0491E02F0FC00A9300E00F3F71
:10142A0050F4ACE8B0E0E02F0E94DA20A981AE17B0
:10143A0010F40F5FF4CFE02F0881229608950E94DE
:10144A00CB2310E020E000E00430A8F40E94DF2063
:10145A00AC91A03081F00E94DF20EC91EA930E94C7
:10146A001123E03041F00E94DF20EC91EA930E94C0
:10147A002923E03009F423C0E12FF22F0E948E23A2
:10148A001E2F2F2F0E94DF20EC91EA930E94172330
:10149A00E03029F00E94DF20EC91E05307C00E945F
:1014AA00DF20EC91EA930E947F23E753A12FB22F0A
:1014BA00F0E0EA2BFB2B1E2F2F2F0F5FC5CFE12F5A
:1014CA00F22F0E94D223259608950A921A92FA922E
:1014DA006A937A938A939A93AA93BA93EA93FA931A
:1014EA00EFB7EA9328970E94CB23E1EEE6BDE0919D
:1014FA006F05E150E0936F05E0918405E150E093B8
:10150A008405E0918705E150E0938705A0916C0579
:10151A00AF5FA0936C05A931C8F0E0E0E0936C05D9
:10152A00E0916D05E150E0936D05E091E804F091DA
:10153A00E904309721F0A8EEB4E00E94E620E09199
:10154A006E05E03019F0E150E0936E05E091CC04AD
:10155A00E03031F0E091CC04E150E093CC04EF5F4D
:10156A00E9B1E095EC7F1E2F103021F0E09178056B
:10157A00E11709F01DC0E0917605F09177053196E3
:10158A00E0937605F0937705EA3FA0E0FA0731F495
:10159A00E2E3E0937A05E093790509C0EC3DA5E022
:1015AA00FA0729F4EAE0E0937A05E09379050CC09A
:1015BA0010937805E0E0E0937605E0937705EFEF86
:1015CA00E0937A05E0937905E0917A05E03011F02D
:1015DA00E15002C0E0917905E0937A05A7ECB4E006
:1015EA000E94EC20F09B0FC0A091C704B091C804E0
:1015FA00E091C304F091C404EA23FB23309711F06D
:10160A00179801C0179AF19B0FC0A091C704B09117
:10161A00C804E091C504F091C604EA23FB2330977D
:10162A0011F0109A01C01098A0911605B0911705F3
:10163A000E94C42358F4A6E1B5E00E94E620E09196
:10164A001105F0E0E951FC4F008126C0EBB5E1FF3E
:10165A0007C0E0911105F0E0E75CFB4F00811CC078
:10166A00A0911405B09115050E94C42358F4A4E171
:10167A00B5E00E94E620E0911105F0E0ED5BFC4F39
:10168A0000810AC0E0911105A0910F05B0911005E3
:10169A00F0E0AE0FBF1F0C91003051F008B913985B
:1016AA00139AE0911105EF5FE0931105E15009C02B
:1016BA00E0E0E09311051198E0E8E8B91398139A6D
:1016CA00119AE0918D05E03009F445C0E13021F42A
:1016DA00EDE30E94F2203DC0E23061F4E0910300A4
:1016EA00E07FE295EF700E94F92008F4095F0E94FA
:1016FA00FE202FC0E33051F4E0910300EF700E9406
:10170A00F92008F4095F0E94FE2023C0E43069F43E
:10171A00E0917105E03019F40E94052103C0EFE25F
:10172A000E94F220E0938D0516C0E53031F40E9444
:10173A000B21EB810E94F2200CC0E63031F40E94AA
:10174A000B21EC810E94F22004C0E73021F40E94B0
:10175A000521E0938D05EAB5E6FF0AC0E091DB00BA
:10176A00E07111F0E0E301C0EEE2EA930E94C808DA
:10177A00E0918305E03009F45FC0E13061F40E9432
:10178A001621E89420F8F798E0E0E0938505EAE06E
:10179A000E941C2151C0E23041F4A0918405A53079
:1017AA0018F4EEE50E941C2147C0E33011F50E94AF
:1017BA002421A0F4E091DB00E07161F40E94292168
:1017CA00E8E2EA1730F4E0E0E0938505EAEF0E94E8
:1017DA001C2103C0E0E0E09385050AC0689420F864
:1017EA000E942F21EAE0E0938405E0E0E09383057C
:1017FA0023C0E43009F50E942421B8F4E091DB000B
:10180A00E07179F00E942921E3E0EA1748F4E091B7
:10181A008605E03011F40E942F21E0E0E093830571
:10182A0003C0E0E0E093850507C0689420F80E94B1
:10183A002F21E0E0E0938305E0918605E03009F48A
:10184A0054C0E13031F4E1E0E09383050E94352190
:10185A004CC0E23069F4E0918305E03041F420FEA7
:10186A0004C0E0E0E093860540C00E943B213DC0F1
:10187A00E330D9F40E94422180F4E091DB00E07168
:10188A0041F40E942921E3E0EA1710F40E943B2167
:10189A0003C0E0E0E093850507C0689420F80E9441
:1018AA002F21E0E0E093860520C0E430F1F40E94A5
:1018BA004221A0F4E091DB00E07161F00E9429214D
:1018CA00E3E0EA1730F40E942F21F79AE0E0E09370
:1018DA00860503C0E0E0E093850507C0689420F818
:1018EA000E942F21E0E0E0938605E0918905E0302F
:1018FA0009F4E9C0E13049F5E0917B05E270B9F0FD
:10190A00E2E3E093CC040E949220E091EE040E946C
:10191A00C420A091D404B091D504EA0FFB1FE09330
:10192A00CE04F093CF04E0918905EF5F0BC0E091FC
:10193A00D604F091D704E459FF4FE093CE04F09314
:10194A00CF04E3E0E0938905BEC0E230D9F4A09168
:10195A00CE04B091CF04AE30E1E0BE0790F4E0913E
:10196A00DB00E47021F4E0918905EF5F08C0ECE147
:10197A00F2E0E093CE04F093CF040E944721E09373
:10198A008905A1C0E33009F5E091DB00E470D1F4E8
:10199A00E0917B05E47051F0E091CE04F091CF0420
:1019AA00309719F4E0E0E09389050BC0E8E1F5E12E
:1019BA00E093CE04F093CF04E0918905EF5FE093C2
:1019CA00890502C00E944C217EC0E43009F5E091ED
:1019DA00DB00E47051F0E8E3F4E0E093CE04F09326
:1019EA00CF04E0918905EF5F10C0A091CE04B091B9
:1019FA00CF04A431E0E0BE0750F4ECE1F2E0E0935A
:101A0A00CE04F093CF040E945321E09389055BC072
:101A1A00E53061F4A091CE04B091CF04A431E0E0A6
:101A2A00BE0718F4E0E0E09389054DC0EC3021F5DB
:101A3A00E091CE04F091CF043097E9F4E0918B0560
:101A4A00E030B9F0E091DB00E47051F4E8E3F4E04F
:101A5A00E093CE04F093CF04E3E0E093890508C055
:101A6A00ECE1F2E0E093CE04F093CF040E94582117
:101A7A0002C00E944C2127C0ED3029F5E091CE0426
:101A8A00F091CF043097F9F4E0918B05E030B9F08A
:101A9A00E091DB00E47051F0E8E3F4E0E093CE0477
:101AAA00F093CF04E5E0E093890508C0ECE1F2E0A9
:101ABA00E093CE04F093CF040E94582104C00E9400
:101ACA005E21E0938905E0918A05E03009F4FDC0C2
:101ADA00E13099F40E946321E093CC040E949220A1
:101AEA00E091EE040E94C420E656F44FE093CE043F
:101AFA00F093CF040E946A21E8C0E23009F5A09170
:101B0A00CE04B091CF04AE30E1E0BE07C0F4E0915C
:101B1A00DB00E27051F4E6E2F6E1E093CE04F093E2
:101B2A00CF04E0918A05EF5F08C0ECE1F2E0E093B0
:101B3A00CE04F093CF040E947021E0938A05C5C0B9
:101B4A00E33009F5A091CE04B091CF04AE30E1E0C4
:101B5A00BE07C0F4E091DB00E27051F0E4EAFFE175
:101B6A00E093CE04F093CF04E0918A05EF5F08C0BA
:101B7A00ECE1F2E0E093CE04F093CF040E94472117
:101B8A00E0938A05A2C0E430F1F4E091CE04F0912A
:101B9A00CF04309769F0E091DB00E17041F0ECE6A8
:101BAA00F0E0E093CE04F093CF040E946A210AC0C9
:101BBA00ECE1F2E0E093CE04F093CF040E945321CB
:101BCA00E0938A0582C0E53059F4E091CE04F091A1
:101BDA00CF04309721F40E947521E0938A0575C0DD
:101BEA00EB3021F5E091CE04F091CF043097E9F47F
:101BFA00E0918B05E030B9F0E091DB00E27051F43E
:101C0A00E6E2F6E1E093CE04F093CF04E3E0E0935A
:101C1A008A0508C0ECE1F2E0E093CE04F093CF0429
:101C2A000E94582102C00E947C214FC0EC3021F54D
:101C3A00E091CE04F091CF043097E9F4E0918B055E
:101C4A00E030B9F0E091DB00E27051F0E4EAFFE144
:101C5A00E093CE04F093CF04E4E0E0938A0508C051
:101C6A00ECE1F2E0E093CE04F093CF040E94582115
:101C7A0002C00E947C2129C0ED3039F5E091CE04E2
:101C8A00F091CF04309709F5E0918B05E030B9F077
:101C9A00E091DB00E17051F0ECE6F0E0E093CE0475
:101CAA00F093CF04E5E0E0938A0508C0ECE1F2E0A6
:101CBA00E093CE04F093CF040E94582106C0EFE3CC
:101CCA00E0937005E5E0E0938A05E0918E05E03047
:101CDA0009F453C0E13081F4A091CE04B091CF044D
:101CEA000E94C42330F4E2EAF0E0E093CE04F093D9
:101CFA00CF040E94832141C0E230C1F4E091CE04B6
:101D0A00F091CF04309789F4E0E0E093CD040E948B
:101D1A006321E093CC040E949220E8E7F9E6E0937D
:101D2A00CE04F093CF040E94832127C0E330C9F484
:101D3A00A091CE04B091CF040E94C42368F4E0912C
:101D4A00DB00E47041F4E8E6FEE2E093CE04F093AF
:101D5A00CF040E94832104C00E947521E0938E055E
:101D6A000CC0E43051F4E091CE04F091CF043097E6
:101D7A0021F40E947521E0938E05E0918F05E030F1
:101D8A0009F47CC0E13099F4E0E0E0938E05A0917B
:101D9A00CE04B091CF040E94C42330F4E2EAF0E00A
:101DAA00E093CE04F093CF040E94892167C0E23009
:101DBA00E1F4E091CE04F091CF043097A9F4E0E089
:101DCA00E093CD04E091DA00E160E093DA00E2E327
:101DDA00E093CC040E949220E8E1F5E1E093CE047E
:101DEA00F093CF040E94892149C0E330E9F4A0911D
:101DFA00CE04B091CF04EEE0F1E0EA17FB0768F4F5
:101E0A00E091DB00E17041F0E4EAFFE1E093CE0407
:101E1A00F093CF040E94892106C0E1E4E0937005A3
:101E2A00E0E0E0938F052AC0E430D9F4E091DB00CA
:101E3A00E47051F0E8E3F4E0E093CE04F093CF04C9
:101E4A00E0918F05EF5F0AC0A091CE04B091CF0454
:101E5A00A431E0E0BE0720F40E945E21E0938F05E2
:101E6A000DC0E53059F4A091CE04B091CF04A4314D
:101E7A00E0E0BE0718F4E0E0E0938F05E091DB00B4
:101E8A00E07291F0A091EB04A33030F4E091EB04FE
:101E9A00EF5FE093EB04E150A091EA04A33019F05C
:101EAA00E0E0E093EA0411C0A091EA04A33030F420
:101EBA00E091EA04EF5FE093EA04E150A091EB04B9
:101ECA00A33019F0E0E0E093EB04A091EA04A33018
:101EDA0021F4A091EB04A33009F00BC0E0E0E093F9
:101EEA00EA04E093EB04E091EC04EF5FE093EC0486
:101EFA00E150A091EC04E0E0EA1770F4E093EC04FE
:101F0A00E0E2FAE0E093E604F093E704E2E3F0E0CB
:101F1A00E093E804F093E904EAB5E1FF06C0739898
:101F2A00739AEAE2E093410503C0EEE2E0934105C9
:101F3A00E091F504E150E093F504E03011F00C94DF
:101F4A006910EDE7E093F504E0917900E093F40479
:101F5A00E0917A00E064E0937A00EAB5E0FF74C0A9
:101F6A00A091F404AF3D38F4E0EDF2E0E09374059B
:101F7A00F09375050FC0E0917405F09175053097DF
:101F8A0031F03197E0937405F093750503C0E3E5EA
:101F9A00E0937005E091F604E03011F00C94201003
:101FAA00A091F404E091F304AE1718F40E948F2173
:101FBA0041C0E091F404A091F304EA1B2E2FE03013
:101FCA0021F4E5E0E093F6042CC0E13021F4E5E0E9
:101FDA00E093F60426C0E23021F4E4E0E093F6044C
:101FEA0020C0E33021F4E4E0E093F6041AC0E430C0
:101FFA0021F4E3E0E093F60414C0E53021F4E3E0D1
:10200A00E093F6040EC0E0E0E093F604283220F4F0
:10201A00E2E0E093F60405C0223318F4E1E0E0932D
:10202A00F6040E949321E091F604E03019F0EAEFF9
:10203A00E093F50408C0E091F604E150E093F60459
:10204A00EF5F0E948F2108C00E948F21E0EDF2E02D
:10205A00E0937405F0937505A091F204E091F10400
:10206A00ED5FAE1780F0A091F204E091F104ED5F0C
:10207A000E94972120F0EDE3E0934A0503C0EEE3C6
:10208A00E0934A050FC0A091F104AD5FE091F2041C
:10209A000E94972120F0EDE3E0934A0503C0ECE3A8
:1020AA00E0934A05E0916E05E03049F4EAE0E21770
:1020BA0018F0E89431F802C0689431F805C06894C1
:1020CA0031F8E3E2E0934A050E94D2232B96E99184
:1020DA00EFBFF991E991B991A99199918991799172
:1020EA006991F9901990099018950A92AA93BA934E
:1020FA00EA93FA93EFB7EA931A930A93EAB5E4FFDD
:10210A000CC0EAB5EF7EEABDE091D004F091D104AB
:10211A00E093CE04F093CF04F49AE091CE04F091C8
:10212A00CF04309711F40C94FD100E949C210E9458
:10213A009C21E091DA00EB7FE093DA00E2E3E0939E
:10214A00CC04AEECB4E00E94E620E091D804F09111
:10215A00D904309739F0A8EDB4E00E94E620309710
:10216A0009F42C9AE091D604F091D704309751F0F3
:10217A00E2E1E093CD04A6EDB4E00E94E6203097B8
:10218A0009F42C98F29B28C0A091CE04B091CF04F8
:10219A00E091CD04F0E0EA17FB0768F4A091CD04C2
:1021AA00E091CA04AE1730F4E091CD04EF5FE093FA
:1021BA00CD04E15010C0A091CE04B091CF04E091BB
:1021CA00CD04F0E0AE17BF0730F4E091CD04E15042
:1021DA00E093CD04EF5F03C0E0E0E093CD04A6EE08
:1021EA00B4E00E94E620309711F4689422F80DC0FA
:1021FA00E0E0E093CD04F498E091CC04E03029F4D7
:10220A00E091DA00E260E093DA00ACE8B1E0E09154
:10221A00CD04F0E0EE0FFF1FEA0FFB1F0E94BB2365
:10222A000E2F1F2FE0938400F093850035FC0AC01F
:10223A00A091CD04A23130F4EBE0F9E0E093840000
:10224A00F0938500A2EDB4E00E94EC20F598E091AD
:10225A009005E03009F4A3C0E13011F00C94761136
:10226A00E091DB00E270B9F1E0E0E0933703E0933C
:10227A003803E0917B05E07159F0E091EF04F091A9
:10228A00F004EC5AF94FE093CE04F093CF0406C061
:10229A00EEE1F6E0E093CE04F093CF04EBB5E2FF73
:1022AA0006C0E0E7F8E0E093CE04F093CF04A091F3
:1022BA00D204B091D304ECEAF4E1EA17FB0750F434
:1022CA00E6E3F0E0E093CE04F093CF040E9470219D
:1022DA00E093900505C0E0919005EF5FE0939005CB
:1022EA005EC0E23001F5689434F8E091DB00E170F9
:1022FA0049F4E0913703F09138033196E0933703BC
:10230A00F0933803E091CE04F091CF04309751F462
:10231A00F59AE0E0E0939005E0E0F0E0E093D20483
:10232A00F093D3043CC0EB30D1F5E091DB00E270CE
:10233A00B9F4E0917B05E07159F0E091EF04F09176
:10234A00F004EC5AF94FE093CE04F093CF0406C0A0
:10235A00EEE1F6E0E093CE04F093CF04E2E01DC094
:10236A00E091CE04F091CF043097C9F4E0918B0547
:10237A00E03049F0ECE1F2E0E093CE04F093CF04D0
:10238A000E9458210CC0E0E0F0E0E093CE04F09304
:10239A00CF04E2E4E0937005E0E0E0939005099150
:1023AA001991E991EFBFF991E991B991A991099030
:1023BA001895AA93BA93EA93FA93EFB7EA930E940D
:1023CA00CA2320E031E00091C6000B3199F4EAB546
:1023DA00E460EABD0E94A221E0E0E0937305E09385
:1023EA00720510E0163028F4A12F0E94A6211F5F63
:1023FA00F9CF5AC0EAB5E2FF2EC0EAB5EB7FEABDD3
:10240A0000937305E02FE13229F1E23519F1E43442
:10241A0009F1E734F9F0EC34E9F0EE34D9F0E035BB
:10242A00C9F0E335B9F0E435A9F0E43799F0EB34B3
:10243A0089F0E73579F0E13469F0E23459F0ED34A6
:10244A0049F0E33439F0E53429F0E53519F0E0E0F4
:10245A00E093730529C0E0917305E030D9F0A091AB
:10246A007205A33198F4B0E0A557BB4F0C930D3019
:10247A0039F4A09172050E94A621EAB5E860EABD86
:10248A00E0917205EF5FE093720503C0E0E0E0932C
:10249A0073050AC0043241F4A22FB32FE6E2F1E237
:1024AA00ED93FC930C94003CEAB5E3FF06C1A091BE
:1024BA007305A23529F457FC02C0689457F8F8C08E
:1024CA00A0917305A33411F0A53409F403C0E0E028
:1024DA00E0939004E0917305E13221F5A0918B0419
:1024EA00A63641F4E0918D05E03019F4E1E0E0937D
:1024FA008D0517C0A0918B04A33629F456FC02C09F
:10250A00689456F80EC0A0918B04A23721F4EBB55B
:10251A00ED7FEBBD06C0A0918B04A13211F40C949F
:10252A000000C6C0E43471F440FC0BC010E0163061
:10253A0030F4A7EFB4E00E94AC211F5FF8CF689493
:10254A0040F8B6C0E73471F441FC0BC010E0163015
:10255A0030F4AAEDB4E00E94AC211F5FF8CF689472
:10256A0041F8A6C0EC3471F442FC0BC010E01630FE
:10257A0030F4A0EEB4E00E94AC211F5FF8CF68945B
:10258A0042F896C0EE3471F443FC0BC010E01630EA
:10259A0030F4ADEFB4E00E94AC211F5FF8CF68942D
:1025AA0043F886C0E03571F444FC0BC010E01630E5
:1025BA0030F4A3E0B5E00E94AC211F5FF8CF689425
:1025CA0044F876C0E33529F455FC02C0689455F8FE
:1025DA006FC0E43571F445FC0BC010E0163030F4DE
:1025EA00A9E0B5E00E94AC211F5FF8CF689445F8D6
:1025FA005FC0E43749F461FC06C0A0918B04A333A1
:10260A0011F4689461F854C0EB3481F446FC0DC0AF
:10261A0010E0163040F4A12FB0E0A458BA4F0E943F
:10262A00B7211F5FF6CF689446F842C0E73529F410
:10263A0047FC02C0689447F83BC0E13429F450FCD7
:10264A0002C0689450F834C0E23429F451FC02C044
:10265A00689451F82DC0E33461F452FC09C010E0CB
:10266A00133120F40E94BE211F5FFACF689452F8FA
:10267A001FC0E53461F460FC09C010E0133120F496
:10268A000E94BE211F5FFACF689460F811C0E53539
:10269A0029F454FC02C0689454F80AC0ED3429F4B1
:1026AA0053FC02C0689453F803C0E0E0E09373055A
:1026BA00E0E0E09373050E94A2210E94D1232496B0
:1026CA00E991EFBFF991E991B991A99118950E9401
:1026DA00C82343EB54E000E010E00430E0E01E07BA
:1026EA0070F45F934F934F5F5F4F0E94C3210E9424
:1026FA00DF08AF91BF91EC930F5F1F4FEECF47EB0F
:10270A0054E000E010E00A30E0E01E0770F45F9346
:10271A004F934F5F5F4F0E94C9210E94DF08AF911C
:10272A00BF91EC930F5F1F4FEECF81D04B9909C039
:10273A00E2E0F0E00E94CF21E3E0F0E00E94CF2146
:10274A0009C0A091B504B091B604A433E2E1BE0772
:10275A0009F420D088D020E031E0A22FB32FE0E0A6
:10276A00F0E0ED93FC937894F09AE0E0F2E0E093E5
:10277A00C304F093C404E9E1E0936F050E94982032
:10278A0008F4FCCFCDD0E4E6E0936E050E94CF2397
:10279A0026960895E1E0E0938205E091B704E0937C
:1027AA00C904E091B804F091B904E093D404F09319
:1027BA00D504E091BA04E093ED04E091BB04E09300
:1027CA00F104E091BC04E093EE04E091BD04F091C1
:1027DA00BE04E093EF04F093F004E091C004E093A8
:1027EA007B050895E091C904E093B704E091D4040D
:1027FA00F091D504E093B804F093B904E091ED04A4
:10280A00E093BA04E091F104E093BB04E091EE0492
:10281A00E093BC04E091EF04F091F004E093BD046E
:10282A00F093BE04E0917B05E093C0040895E2E0D2
:10283A00E093C904E4E2F2E1E093D404F093D5040E
:10284A00E0E0E093ED04E1E9E093F104E0E1E093F4
:10285A00EE04E0E0F0E0E093EF04F093F004E0E14E
:10286A00E0937B0508950A930E94D521E0E0F0E009
:10287A00E093CE04F093CF04E2E4E093CA04F29A20
:10288A00E0E0E093CD04E093EA04E093EB04E09304
:10289A00EC04E0E2FAE0E093E604F093E704EDE703
:1028AA00E093F504E091F1040E94A120E093F3047F
:1028BA00E0E0E0931105E09312050E94DB21E0932A
:1028CA0033030E94EB0800E0003540F4A02FB0E08B
:1028DA00AD5BBC4FE0E2EC930F5FF6CFE0E0E09334
:1028EA00930300E0003540F4A02FB0E0A951BC4F9B
:1028FA00E0E2EC930F5FF6CFE0E0E093370400E00C
:10290A00003528F4A02F0E94E3210F5FF9CFE0E001
:10291A00E0938904EDE7F2E00E94A5200991089569
:10292A00ECE3E0936D05E0916D05E03029F0E0916C
:10293A00F404E03009F4F7CFA091F404AC3318F4AE
:10294A00E3E5E0937005E1E0E0938605E091860512
:10295A00E030E1F7F79907C0E1E0E0938605E091FE
:10296A008605E030E1F720FE03C0E4E5E093700558
:10297A00F79903C0E4E5E0937005E2E3E093CC0441
:10298A000E949220E091DB00E17041F0E091DB00CF
:10299A00E27021F0E091DB00E47009F40FC0E6E494
:1029AA00F5E0E093CE04F093CF04A091CE04B09169
:1029BA00CF04EEE0F1E0EA17FB07B8F3E091DB00A1
:1029CA00E17041F0E091DB00E27021F0E091DB0080
:1029DA00E470E1F5E8E8FDE1E093D004F093D10476
:1029EA000E949D20F49AEAB5E4FDFDCFE091DB0058
:1029FA00E47049F0A091CE04B091CF04EEE0F1E08A
:102A0A00EA17FB0708F001C0F1CFE0EAF2E3E0932E
:102A1A00D004F093D1040E949D20F49AEAB5E4FD13
:102A2A00FDCFE091DB00E47049F4A091CE04B091AF
:102A3A00CF04EEE0F1E0EA17FB0708F001C0F1CF9E
:102A4A00E8E3F4E0E093CE04F093CF04E091CE04FF
:102A5A00F091CF043097D1F7E091DB00E17041F0BB
:102A6A00E091DB00E27021F0E091DB00E47019F400
:102A7A00E6E5E09370050E94D1200E949321089513
:102A8A000E94CA234CD5E0911605F091170530979C
:102A9A0019F4EBB5E1FF01C0F5CF4C9907C1E091FC
:102AAA001305EF5FE0931305E130B1F4ECE7F3E0CF
:102ABA00FA93EA93E2EDF2E00E94E921EDE8F3E00D
:102ACA00FA93EA930E9437236DD4E5E9F3E0E093A1
:102ADA000F05F0931005DAC0E230B1F4EEEDF3E041
:102AEA00FA93EA93E2EDF2E00E94E921EFEEF3E0D5
:102AFA00FA93EA930E94372369D4E5E9F3E0E09375
:102B0A000F05F0931005C2C0E330B1F4E0E4F4E03D
:102B1A00FA93EA93E2EDF2E00E94E921E1E5F4E0BA
:102B2A00FA93EA930E94372360D4E5E9F3E0E0934D
:102B3A000F05F0931005AAC0E430B1F4E2EAF4E01C
:102B4A00FA93EA93E2EDF2E00E94E921E3EBF4E082
:102B5A00FA93EA930E9437235ED4E5E9F3E0E0931F
:102B6A000F05F093100592C0E530B1F4E5E0F5E009
:102B7A00FA93EA93E2EDF2E00E94E921E6E1F5E058
:102B8A00FA93EA930E943723B4D4E5E9F3E0E09399
:102B9A000F05F09310057AC0E630B9F4E7E6F5E0E0
:102BAA00FA93EA93E2EDF2E00E94E921E8E7F5E020
:102BBA000E94F621E07141F0E6ECF3E0FA93EA9321
:102BCA00E9ECF5E00E94032261C0E73011F00C94B1
:102BDA004A164F995AC0E1EDF5E0FA93EA93E2ED0D
:102BEA00F2E00E94E921E2EEF5E00E94F621E270AD
:102BFA0021F4E0917B05E47009F007C0E9ECF3E009
:102C0A00FA93EA93E3E3F6E026C0E0917B05E270EB
:102C1A0021F0E0917B05E47009F007C0E9ECF3E0EC
:102C2A00FA93EA93E8E3F6E016C0E0917B05E270D6
:102C3A0021F4E0917B05E47009F407C0E9ECF3E0C4
:102C4A00FA93EA93EDE3F6E006C0E9ECF3E0FA93CF
:102C5A00EA93E2E4F6E0FA93EA930E940922F799EA
:102C6A000AC0E5E9F3E0FA93EA93E7E4F6E0FA93B7
:102C7A00EA930E940D224F9BFECFE7E0E0936F0597
:102C8A000E94982008F4FCCF01C071D3EFE0E093D2
:102C9A006F050E94982008F4FCCF4C9BFECFEFE012
:102CAA00E0936F050E94982008F4FCCFA0911305C9
:102CBA00E0E0EA1720F4A0911305A73009F409C04F
:102CCA00E091DB00E17011F056FE03C050D3E894A6
:102CDA0056F8A0911305E0E0EA1740F4A091130515
:102CEA00A63021F0A0911305A73009F415C04B991D
:102CFA0013C03DD3E89456F8E2E0E0936F050E94D2
:102D0A00982008F4FCCF4B9BFECFE2E0E0936F05DE
:102D1A000E94982008F4FCCFA0911305A63011F068
:102D2A000C94E5164D994CC0EDE4F6E0FA93EA935B
:102D3A00EEE5F6E0FA93EA93EEEEF2E0FA93EA931E
:102D4A000E94EC090E941122E093B504F093B604A4
:102D5A000E94F71323EB34E000E010E00430E0E0D7
:102D6A001E0748F40E94C3210E941A222F5F3F4F78
:102D7A000F5F1F4FF3CF27EB34E000E010E00A307B
:102D8A00E0E01E0748F40E94C9210E941A222F5F20
:102D9A003F4F0F5F1F4FF3CF0E94DB21E0931305D4
:102DAA00E2E0E0936F050E94982008F4FCCF4D9B67
:102DBA00FECFE2E0E0936F050E94982008F4FCCF72
:102DCA00A3E1B5E0EC91E13011F00C942E174A9989
:102DDA001EC0A091C904A03128F4E091C904EF5F94
:102DEA00E093C9040E9420220E94982008F4FCCF94
:102DFA004A9904C0E0917A05E03009F401C0F8CF9D
:102E0A00E2E0E0936F050E94982008F4FCCF4E9907
:102E1A001FC0A091C904E0E0EA1728F4E091C904B0
:102E2A00E150E093C9040E9420220E94982008F4ED
:102E3A00FCCF4E9904C0E0917A05E03009F401C054
:102E4A00F8CFE2E0E0936F050E94982008F4FCCFE7
:102E5A0084C2E23011F00C9474174A991EC0A091F2
:102E6A00ED04AE3128F4E091ED04EF5FE093ED0458
:102E7A000E9426220E94982008F4FCCF4A9904C096
:102E8A00E0917A05E03009F401C0F8CFE2E0E0937E
:102E9A006F050E94982008F4FCCF4E991FC0A0919C
:102EAA00ED04E0E0EA1728F4E091ED04E150E09344
:102EBA00ED040E9426220E94982008F4FCCF4E9925
:102ECA0004C0E0917A05E03009F401C0F8CFE2E0ED
:102EDA00E0936F050E94982008F4FCCF3EC2E330CD
:102EEA0011F00C94BC174A991FC0A091EE04AE31A0
:102EFA0030F4E091EE04EF5FE093EE04E1500E94BB
:102F0A002C220E94982008F4FCCF4A9904C0E09130
:102F1A007A05E03009F401C0F8CFE2E0E0936F05EA
:102F2A000E94982008F4FCCF4E9920C0A091EE048C
:102F3A00EAE0EA1730F4E091EE04E150E093EE049F
:102F4A00EF5F0E942C220E94982008F4FCCF4E9931
:102F5A0004C0E0917A05E03009F401C0F8CFE2E05C
:102F6A00E0936F050E94982008F4FCCFF6C1E43084
:102F7A0011F00C9408184A9921C0A091EF04B0915D
:102F8A00F004A436E0E0BE0724F4AFEEB4E00E94F9
:102F9A00EC200E9432220E94982008F4FCCF4A9921
:102FAA0004C0E0917A05E03009F401C0F8CFE2E00C
:102FBA00E0936F050E94982008F4FCCF4E9922C036
:102FCA00A091EF04B091F004ECE9FFEFEA17FB07D8
:102FDA0024F4AFEEB4E00E94E6200E9432220E945E
:102FEA00982008F4FCCF4E9904C0E0917A05E030AD
:102FFA0009F401C0F8CFE2E0E0936F050E9498203F
:10300A0008F4FCCFAAC1E53011F00C945A184A9979
:10301A0024C0A091D404B091D504AC3FE2E1BE072C
:10302A0038F4A4EDB4E00E94B723F696ED93FC932E
:10303A000E9438220E94982008F4FCCF4A9904C0C2
:10304A00E0917A05E03009F401C0F8CFE2E0E093BC
:10305A006F050E94982008F4FCCF4E9925C0A091D4
:10306A00D404B091D504E0EEF0E1EA17FB0738F496
:10307A00A4EDB4E00E94B723F697ED93FC930E9467
:10308A0038220E94982008F4FCCF4E9904C0E0919F
:10309A007A05E03009F401C0F8CFE2E0E0936F0569
:1030AA000E94982008F4FCCF58C1E63079F54A9975
:1030BA002CC0E0917B05E07159F0E6ECF3E0FA935D
:1030CA00EA93EFE6F6E00E9403220E943E220DC038
:1030DA00E0917B05E061E0937B05E6ECF3E0FA938F
:1030EA00EA93E9ECF5E00E940322E2E0E0936F053F
:1030FA000E94982008F4FCCF4A9BFECFE2E0E093BE
:10310A006F050E94982008F4FCCF27C1E73011F020
:10311A000C94B2194A994FC0E2E0E0936F050E94FD
:10312A00982008F4FCCF4A9BFECFE2E0E0936F05BB
:10313A000E94982008F4FCCF4A9B2BC00E9444228C
:10314A00F79B0EC0E1E0E0938305E0918305E03050
:10315A00E1F7E5E9F3E0FA93EA93E7E4F6E00DC074
:10316A00E1E0E0938605E0918605E030E1F7E5E9E4
:10317A00F3E0FA93EA93E7E7F6E0FA93EA930E9418
:10318A000D22EBE4E0936F050E94982008F4FCCF2F
:10319A00D3CF0E944822E2E0E0936F050E94982074
:1031AA0008F4FCCF4A9BFECFE2E0E0936F050E9451
:1031BA00982008F4FCCF4E992DC00E944422E09139
:1031CA00BE03E43449F40E942F21EDEBF3E0FA93B5
:1031DA00EA93EDE7F6E008C00E941621EDEBF3E072
:1031EA00FA93EA93E3E8F6E0FA93EA930E940D224F
:1031FA00E2E0E0936F050E94982008F4FCCF4E9B12
:10320A00FECFE2E0E0936F050E94982008F4FCCF1D
:10321A000E9448224F9927C0E091C403E43441F444
:10322A002C98E3ECF3E0FA93EA93E9E8F6E007C0B6
:10323A002C9AE3ECF3E0FA93EA93EFE8F6E0FA93D8
:10324A00EA930E940D22E2E0E0936F050E94982023
:10325A0008F4FCCF4F9BFECFE2E0E0936F050E949B
:10326A00982008F4FCCF4B9958C0E0917B05E27096
:10327A0021F4E0917B05E47009F00CC00E944C2215
:10328A00E260E0937B05E9ECF3E0FA93EA93E8E382
:10329A00F6E02FC0E0917B05E27021F0E0917B051A
:1032AA00E47009F00CC00E944C22E460E0937B05B4
:1032BA00E9ECF3E0FA93EA93EDE3F6E01AC0E09161
:1032CA007B05E27021F4E0917B05E47009F409C002
:1032DA000E945222E9ECF3E0FA93EA93E2E4F6E080
:1032EA0008C00E945822E9ECF3E0FA93EA93E3E378
:1032FA00F6E0FA93EA930E940922E2E0E0936F056E
:10330A000E94982008F4FCCF4B9BFECFE2E0E093AA
:10331A006F050E94982008F4FCCF4D991EC0E2E385
:10332A00E093CC040E949220EFEFFFEFE093D004E9
:10333A00F093D1040E949D20F49AE2E0E0936F0595
:10334A000E94982008F4FCCF4D9BFECFE2E0E09368
:10335A006F050E94982008F4FCCFA0911305E0E0C5
:10336A00EA1708F48FCB0E94D123249608950E946D
:10337A00DB21E0931305E5E0F0E0E0931405F09318
:10338A0015052C98F79907C0E1E0E0938605E091CE
:10339A008605E030E1F7ECE6F0E0E093CE04F09346
:1033AA00CF0408950E945E22E5E9F6E00E946322B6
:1033BA00FF27662777270E94BF2384E00E94042004
:1033CA002896EDEBF3E00E946822A7C00E945E22D5
:1033DA00E6EAF6E00E94722284E00E94042028961F
:1033EA00EDEBF3E00E94682298C00E945E22ECEBAB
:1033FA00F6E0FA93EA93E091EE04FF27662777272F
:10340A000E94BF2384E00E9404202896EDEBF3E09B
:10341A000E94682282C0A8974A9911C0FE01FA93B5
:10342A00EA93E4EDF6E0FA93EA93E091EF04F0917F
:10343A00F0040E9497230E94BF2384E052C04E9951
:10344A0011C0FE01FA93EA93E6EEF6E0FA93EA93E4
:10345A00E091EF04F091F0040E9497230E94BF23A9
:10346A0084E03FC0A091EF04B091F0040E94C4230D
:10347A008CF4FE01FA93EA93E4EDF6E0FA93EA9308
:10348A00E091EF04F091F0040E9497230E94BF2379
:10349A0084E027C0A091EF04B091F00410978CF457
:1034AA00FE01FA93EA93E6EEF6E0FA93EA93E091E4
:1034BA00EF04F091F0040E9497230E94BF2384E056
:1034CA0010C0FE01FA93EA93E8EFF6E0FA93EA9362
:1034DA00E091EF04F091F0040E9497230E94BF2329
:1034EA0084E00E9404202896EDEBF3E00E94682213
:1034FA0014C00E945E22ECEBF6E0FA93EA93A091E4
:10350A00D404B091D5040E94802284E00E94042051
:10351A002896EDEBF3E00E946822A8960895289772
:10352A0082E0A2E0B0E0EEE3F2E00E94D6230E943D
:10353A00C823E0910500A0910400EA2BA09106009F
:10354A00EA2B21F40E94CF232E96089557FE32C00B
:10355A000E94892221F4A0918D05A03009F012C0A1
:10356A00EBB5E0FF06C0EAE0F7E0FA93EA9380E001
:10357A0005C0EDE0F7E0FA93EA9380E00E94172095
:10358A00229616C0A0918B04A03359F4EBB5EE7FB6
:10359A00EBBDE0917105E0937005E0E0E093710501
:1035AA0007C0A0918B04A13319F4EBB5E160EBBD20
:1035BA00E89457F840FE28C0E7EFF4E00E94912211
:1035CA0021F4A0918D05A03009F009C0E0E1F7E0EF
:1035DA000E94722284E00E941720269613C0E7EF09
:1035EA00F4E00E949722E8EBFBE0E217F30710F4FD
:1035FA0028EB3BE0A22FB32FE4E6F0E00E94A423DD
:10360A00E093ED04E89440F841FE39C0EAEDF4E0B5
:10361A000E94912221F4A0918D05A03009F00EC0DC
:10362A00E0E1F7E00E946322FF27662777270E94DE
:10363A00BF2384E00E94172026961FC0EAEDF4E01B
:10364A00FA93EA930E942520ED87AD85E2E1EA1715
:10365A0008F4ED87E0E0EA87AA85A63158F4A8E2E3
:10366A00B2E0EA850E94DA20AD85EA1718F40E94D2
:10367A009E22F2CFEA85E093C904E89441F842FE1B
:10368A0036C0E0EEF4E00E94912221F4A0918D056B
:10369A00A03009F00FC0E0E1F7E0FA93EA93A091B5
:1036AA00D404B091D5040E94802284E00E9417209D
:1036BA0026961BC0E0EEF4E00E9497222035E0E057
:1036CA003E0710F420E530E0EAE5F0E0E217F30700
:1036DA0010F42AE530E0A22FB32FE6E3F0E00E94CF
:1036EA009C23E093D404F093D504E89442F843FE73
:1036FA0031C0EDEFF4E00E94912221F4A0918D05F2
:10370A00A03009F010C0E0E1F7E0FA93EA93E09103
:10371A00EE04FF27662777270E94BF2384E00E94D2
:10372A001720269615C0EDEFF4E00E9497222A3062
:10373A00E0E03E0710F42AE030E0EEE1F0E0E217C4
:10374A00F30710F42EE130E0E22FF32FE093EE04BA
:10375A00E89443F844FE36C0E3E0F5E00E94912283
:10376A0021F4A0918D05A03009F011C0E4E1F7E041
:10377A00FA93EA93E091EF04F091F0040E94972300
:10378A000E94BF2384E00E941720269619C0E3E016
:10379A00F5E0FA93EA930E9425200E2F1F2F0C3989
:1037AA00EFEF1E0714F40CE91FEFE4E6F0E0E01770
:1037BA00F10714F404E610E00093EF041093F00408
:1037CA00E89444F845FE38C0E9E0F5E00E94912209
:1037DA0021F4A0918D05A03009F010C0E0E1F7E0D6
:1037EA00FA93EA93E091F104FF27662777270E946C
:1037FA00BF2384E00E94172026961CC0E9E0F5E06A
:10380A000E9497222436E0E03E0710F424E630E0D6
:10381A00E4EBF0E0E217F30710F424EB30E0E22FD8
:10382A00F32FE093F104E091F104EA930E94120A63
:10383A00E093F304E89445F861FE18C0E091F404BB
:10384A00EA930E94080AE093F204E0E1F7E0FA93AF
:10385A00EA93E091F204FF27662777270E94BF23A5
:10386A0084E00E9417202696E89461F846FE55C027
:10387A00ECE7F5E00E94912221F4A0918D05A03099
:10388A0009F011C0E8E1F7E0FA93EA93E0917B05C9
:10389A00E17FFF27662777270E94BF2384E00E94E3
:1038AA001720269638C0E0917B05EB87E0917E05CC
:1038BA00EB33B9F4E0E0E0937E050E94A222EC87A4
:1038CA00E0917F05E03331F4EC85E095AB85EA239E
:1038DA00EB8706C0E13321F4EC85AB85EA2BEB8755
:1038EA0003C00E94A222EB870E94A822EB85E17006
:1038FA000E94AE22E0917B05E17021F0EEE2E093B6
:10390A00420503C0EDEEE09342050E943E22EB859C
:10391A00E0710E94AE22E89446F847FE3BC00E943E
:10392A00892221F4A0918D05A03009F011C0F79BDE
:10393A0006C0EDE0F7E0FA93EA9380E005C0EAE01A
:10394A00F7E0FA93EA9380E00E941720229620C0BB
:10395A00A0918B04A03389F4E1E0E0938605E0911D
:10396A008605E030E1F7F79907C0E1E0E0938605C4
:10397A00E0918605E030E1F70BC0A0918B04A133FA
:10398A0039F4E1E0E0938305E0918305E030E1F763
:10399A00E89447F850FE26C00E94892221F4A0919B
:1039AA008D05A03009F011C02C9B06C0EAE0F7E0B3
:1039BA00FA93EA9380E005C0EDE0F7E0FA93EA9320
:1039CA0080E00E94172022960BC0A0918B04A1339D
:1039DA0011F42C9A05C0A0918B04A03309F42C98F9
:1039EA00E89450F851FE30C00E94892221F4A09137
:1039FA008D05A03009F013C0E0917B05E17031F02C
:103A0A00EAE0F7E0FA93EA9380E005C0EDE0F7E038
:103A1A00FA93EA9380E00E941720229613C0A0919D
:103A2A008B04A03331F40E94A822EDEEE093420504
:103A3A0009C0A0918B04A13329F40E94D521EEE29A
:103A4A00E0934205E89451F852FE7CC00E94B422E9
:103A5A0041F4E091A004EB3321F4E091B104E030A9
:103A6A0009F06EC0A0919F04A03399F5E7EEF3E048
:103A7A00FA93EA93E1EAF4E00E94BE22E091160585
:103A8A00F09117053097F9F4EBB5E1FF07C0EFE0C5
:103A9A00F4E0FA93EA93E1E6F4E011C0E091130549
:103AAA00E03039F0EFE0F4E0FA93EA93EDEBF3E07B
:103ABA0006C0EFE0F4E0FA93EA93E0E4F5E0FA9363
:103ACA00EA930E94C422ECEDF5E0E0931605F09328
:103ADA001705A0919F04A13399F5EFE0F4E0FA935A
:103AEA00EA93E1EAF4E00E94BE22E0911605F09121
:103AFA0017053097F9F4EBB5E1FF07C0E7EEF3E0FD
:103B0A00FA93EA93E9E3F4E011C0E0911305E03097
:103B1A0039F0E7EEF3E0FA93EA93E5E9F3E006C059
:103B2A00E7EEF3E0FA93EA93E8E1F5E0FA93EA9331
:103B3A000E94C422ECEDF5E0E0931605F093170518
:103B4A00E89452F860FE49C00E94B42241F4E09120
:103B5A00A004EB3321F4E091B104E03009F038C05D
:103B6A00A0919F04A033D9F4E9E3F4E0FA93EA932D
:103B7A00E1EAF4E00E94BE22EBB5E1FD10C0E0E00C
:103B8A00EA87AA85A03158F4EA85E85DF0E0E75CA7
:103B9A00FB4FDF01E0E2EC930E949E22F2CFA0915C
:103BAA009F04A133A9F4E1E6F4E0FA93EA93E1EA87
:103BBA00F4E00E94BE22EBB5E1FD0AC0E0E0EA872C
:103BCA00AA85A03128F40E94E3210E949E22F8CF00
:103BDA00EBB5E260EBBDE89460F853FE77C00E9453
:103BEA00892221F4A0918D05A03009F035C0E09119
:103BFA007B05E27021F0E0917B05E47009F406C0D0
:103C0A00EEE1F7E0FA93EA9380E022C0E0917B05C7
:103C1A00E27021F4E0917B05E47009F006C0EDE062
:103C2A00F7E0FA93EA9380E013C0E0917B05E27033
:103C3A0031F0EAE0F7E0FA93EA9380E009C0E09114
:103C4A007B05E47041F0E1E2F7E0FA93EA9380E061
:103C5A000E941720229638C0E0918B04E03319F4B1
:103C6A000E94582231C0E13331F40E944C22E260B2
:103C7A00E0937B0529C0E23331F40E944C22E460D0
:103C8A00E0937B0521C0E33319F40E9452221CC041
:103C9A00E43361F4689432F8E1E2E0934305EEE735
:103CAA00E0934405E1E0E0938E050EC0E53361F44C
:103CBA00689432F8E1E2E093430536F8EFE7E093DF
:103CCA004405E1E0E0938F05E89453F855FE2EC0D1
:103CDA000E941122E093B504F093B6040E94F713F0
:103CEA00E3EBF4E0EE83FF8340E050E04430E0E0B1
:103CFA005E0740F4E42FF52F30960E94C8224F5FEA
:103D0A005F4FF4CFE7EBF4E0EE83FF8340E050E04F
:103D1A004A30E0E05E0740F4E42FF52F70960E94E7
:103D2A00C8224F5F5F4FF4CFE89455F854FE17C08E
:103D3A00EBE8F4E0FA93EA930E944223E130A0E030
:103D4A00FA0721F4A0918B04A43209F008C0A885CF
:103D5A00B985E6E2F1E2ED93FC930C94003C0E94F3
:103D6A00CF232E960895E091C000E072E1F3E88136
:103D7A00E093C60021960895A881B9810E94B723CD
:103D8A00309731F00E94EC203197AA81A08304C0B9
:103D9A00EA81EA930E94B81E2396089526970E9404
:103DAA00C82300E0E889F9893196E88BF98B3197C5
:103DBA00E4913E2FE03011F40C940020E02FE03023
:103DCA0039F4353211F401E002C00E94D62212C140
:103DDA00E130B1F4353221F40E94D62200E00AC162
:103DEA0002E050E010E03D3211F411E003C13B3231
:103DFA0011F45BE2FFC0303211F450E2FBC002C0A2
:103E0A00E23039F440E003E0303311F41068F2C0D4
:103E1A0004C0E33011F00C94FF1F303310F03A3332
:103E2A0008F009C0A42FEAE0EA9FE02D4E2FE32F05
:103E3A00E0534E0FDFC0E32FE33631F40E94DD2258
:103E4A00EC910E94E422D5C0E33741F40E94DD22BE
:103E5A000E94EB220E9442230E2F0AC0E03761F42F
:103E6A000E94DD220E94EB220E944C230E2F186032
:103E7A0012601F7720E038C0E43611F0E93611F4F9
:103E8A00146002C0E53731F4E0E4F2E0EE83FF8328
:103E9A0005E00DC0E83511F4186004C0E83711F0E8
:103EAA000C94FE1FEAE4F2E0EE83FF8304E012FFC3
:103EBA0015C00E94DD220E94B723EA87FB87AA85E4
:103ECA00BB8510972CF40E948A23EA87FB875DE260
:103EDA00503011F00F5F01C01B7F06C00E94DD2227
:103EEA000E94B723EA87FB8710FD11C0041778F4F4
:103EFA0017FF08C012FF04C01B7F352F015001C0F5
:103F0A0030E301C030E20E94D6224150EFCF202F89
:103F1A0011FF1AC02030B9F013FF08C0EE81FF81EB
:103F2A003196EE83FF833197E49105C0AE81BF815C
:103F3A00ED91AE83BF83EA930E94F222403009F0EA
:103F4A0041502150E7CF4CC030E3EE81FF813296D9
:103F5A00EE83FF8332970E94BB23E887F987AA85FD
:103F6A00BB85AE17BF0720F03F5FAE1BBF0BC9F77B
:103F7A00AA87BB87E9E3E31728F413FF02C0395F76
:103F8A0001C0395D14FD1EC0E0E3E31730F0A885D7
:103F9A00B985A130E0E0BE0711F410610AC04217EA
:103FAA0010F010FF01C013C030E217FF0BC030E35E
:103FBA00106112FF07C01B7F5A930E94F222403001
:103FCA0009F041500E94D622403009F04150215058
:103FDA00A885B985E1E0F0E0EA17FB0708F4B4CF59
:103FEA0010FF07C0403029F04150E0E20E94E4226D
:103FFA00F9CF00E0D7CE0E94CF2362960895FF92B0
:10400A00F82E0E94F822DE0116960E9486230E944C
:10401A00B723EA83FB830E940123AA81BB81E0E0E4
:10402A00EC9309C0FF92F82E0E94F822E0E0EA839E
:10403A00EB830E940123198108812496FF90089539
:10404A00B981A881EC91EA930E941F23EE2311F013
:10405A001196F8CFE894EC91ED3211F4689402C00D
:10406A00EB3209F4119666277727EC91EA930E94BE
:10407A001723EE2381F0E62FF72F660F771F660FBF
:10408A00771F6E0F7F1F660F771FED91FF27E05393
:10409A006E0F7F1FEACFE62FF72F1EF4E095F095FB
:1040AA00319622960895A991B991E991F99130969C
:1040BA002AF4E095F09531966DE26D93E89480E1EB
:1040CA0097E20DD088EE93E00AD084E6992707D0CC
:1040DA008AE005D06E2F10D066276C930895662764
:1040EA00E817F90720F06395E81BF90BC9F766236F
:1040FA0011F416F008956894605D6D930895FA932B
:10410A00EA93FE013296FA93EA93E3E0EA930C9477
:10411A005723E0E1EA930C946B23E091DA00ED7FF8
:10412A00E093DA000895A0916F05E0E0EA17089598
:10413A00EAB5E061EABD0895ED5FEA930C94120ACC
:10414A00FA93EA93EAE7F0E0FA93EA93E4EFF1E00C
:10415A00FA93EA930C94EC09E0918805EF5FE093F7
:10416A0088050895E1E0E0938305F6CFE091DA004F
:10417A00E77FE093DA00E1E0E09386050895F0E056
:10418A00A6E3B0E00E949C230895E091C904F0E000
:10419A00EA0FFB1FE4910895EAB5E160EABD0895CC
:1041AA00E0E0E0939005EEE20895F0E0EA0FFB1FED
:1041BA00E4910895E02FAB81BC81F0E0AE0FBF1F00
:1041CA0008950E94B7233197ED93FC9308950E94B6
:1041DA00B7233196ED93FC930895EA930E94C80899
:1041EA00E0918D05EF5F0895E0630E2FE9E3E01794
:1041FA0008950A930E94C808E0918D05EF5F08951B
:10420A00EDE0EA930E94C808E0E00895E0917105A4
:10421A00F0E0FA93EA93FE013596FA93EA930C9446
:10422A005820E091DA00E061E093DA000895E09323
:10423A008405E0918305EF5FE09383050895A091DB
:10424A008405E5E0EA170895A0918505AF5FA0937C
:10425A0085050895E091DA00EF7EE093DA0008958B
:10426A00E0918605EF5FE09386050895E0E0E0932C
:10427A008505E9E1E0938705F3CFA0918705E5E09D
:10428A00EA170895EAE0E0938B05ECE00895E1E48B
:10429A00E0937005E0E0E09389050895EAE0E09391
:1042AA008B05EDE00895E0918B05E150E0938B05D5
:1042BA000895E0E4E0937005E0E00895E091DA0003
:1042CA00EE7FE093DA00E2E30895E0918A05EF5F7A
:1042DA00E0938A050895EAE0E0938B05EBE0089500
:1042EA00E091DA00E160E093DA00E0E00895E1E4C9
:1042FA00E0937005E5E0E0938A050895E0918E0564
:10430A00EF5FE0938E050895E0918F05EF5FE093EC
:10431A008F050895EAB5ED7FEABD0895EAB5E26032
:10432A00EABD0895AE1B2A2FEAE0E2170895E0914C
:10433A00DA00E460E093DA000895EAB5E77FEABDBF
:10434A000895B0E0A557BB4FE0E0EC930895E12F44
:10435A00F0E0AE0FBF1FE12FF0E0E557FB4FE08121
:10436A00EC930895E12FF0E0E557FB4FE081EC93E1
:10437A000895A12FB0E0A156BB4FF4CFE02FF12F43
:10438A003096FA93EA930895E02FF12F7096FA93F4
:10439A00EA930895FA93EA93E0E0EA930C94D10839
:1043AA00E0917B05E160E0937B050895E8E1F5E0A3
:1043BA00E0930F05F0931005E0E00895B0E0A75CE4
:1043CA00BB4FE0E2EC930895FA93EA93EEEEF2E043
:1043DA00FA93EA930E94EC09E5E9F3E0FA93EA9387
:1043EA000895FA93EA930E943723E5E9F3E0E0930C
:1043FA000F05F0931005E0917B050895FA93EA936F
:10440A00E7E0EA930C946B23E4E0EA930C946B23C1
:10441A00E5E0EA930C946B23E1E4FCE4E093B30453
:10442A00F093B404E4E3F2E10895A22FB32FEC91E0
:10443A00EA930C94D1080E94D719E2E0E0936F0541
:10444A0008950E94EB19E2E0E0936F0508950E9437
:10445A00FA19E2E0E0936F0508950E94101AE2E06B
:10446A00E0936F0508950E947E1AE2E0E0936F05DB
:10447A000895E0917B05EF7EE0937B050895EAB508
:10448A00E064EABD0895EAB5EF7BEABD0895E091DC
:10449A007B05E97FE0937B050895E0917B05E66063
:1044AA00E0937B050895E0917B05E97FE0937B0526
:1044BA000895A897FE01FA93EA930895FA93EA9366
:1044CA00A8E2B2E062CEFA93EA93FE013296FA9338
:1044DA00EA93E0E1EA930C945723FA93EA93E09182
:1044EA00ED04F0E0A4E6B0E00E949C23662777275B
:1044FA000E94BF230895E6E3F0E00E94A423662702
:10450A0077270E94BF230895EBE8F4E0FA93EA9331
:10451A000E94422330970895FA93EA930E94422315
:10452A0030970895FA93EA930E9425202E2F3F2F61
:10453A000895EA85EF5FEA870895ECE7F5E0FA93D4
:10454A00EA930C94240AE0917B05EE7FE0937B05C5
:10455A000895A0917B05EA2BE0937B050895EFE986
:10456A00F4E0FA93EA930E944223E231A0E0FA07C8
:10457A000895FA93EA93E0E1EA930C945723E0E171
:10458A00EA930C945723FA93EA93A885B985EC9198
:10459A00EA930E94D108EE81FF813196EE83FF8370
:1045AA0008953A93ED85FE85FA93EA930C94C11E19
:1045BA00AE85BF851497AE87BF8714960895EA9390
:1045CA00ED85FE85FA93EA930C94C11E0E94B723E7
:1045DA00EE83FF83FA93EA930895ED85FE85FA93B5
:1045EA00EA930C94C11E22971A930A93DE010E9441
:1045FA0086230A2F1B2F0895DE0114960E94862314
:10460A000E94B723FA93EA931A930A93FE01369605
:10461A00FA93EA930C94D31EE1E0F991F03808F08A
:10462A00EE270895E1E0F991F03310F0FA3308F03B
:10463A00EE270895E1E0F991F03229F0F93010F00F
:10464A00FE3008F0EE270895E1E0F991F05340F0CA
:10465A00FA3038F0FF75F750FA3010F0F03108F000
:10466A00EE270895E991F991A991B991CD010590A3
:10467A000D920020E1F7FC010895A991B991EE2766
:10468A00FF276D91662311F03196FBCF0895AA2773
:10469A00BB27E991F9910590002011F01196FBCF03
:1046AA00FD0108957991E991F991A991B991CD0105
:1046BA00772351F07A9561916D936623C9F7772331
:1046CA0019F07A956D93FBCFFC0108956991E991F0
:1046DA00F991A991B991CD01662351F06A95059096
:1046EA000D920020C9F7662319F06A950D92FBCF47
:1046FA00FC010895E991E13618F0EB3708F4E0522D
:10470A0008950024AF0DB01D0895E095F0953196F7
:10471A000895EE0FFF1FEE0FFF1FEE0FFF1FEE0FA4
:10472A00FF1F08956F2F660F660B762F0895FA9F65
:10473A00F02DEB9FF00DEA9FE02DF10D0895002476
:10474A00112490E1AA0FBB1F001C111C0E1A1F0A8C
:10475A0018F40E0E1F1E01C0A1609A9599F7FD016B
:10476A00D0010895ED91FC91119708950590F49167
:10477A00E02D08957A936A93FA93EA9308950024B0
:10478A000A160B0608955A934A933A932A931A9350
:10479A000A9308955D814C813B812A8119810881A0
:1047AA000895AC0FBD1F05900D928A95E1F7089503
:00000001FF
